:0400000012C08BC0DF
:10000400FDCFCAC0FBCFFACFF9CFF8CFF7CFF6CFE9
:1000140000000000010002001400020005001600A8
:100024000000F894EE27ECBBE5BFF8E1A4B7A77F86
:10003400A4BFF1BDE1BD8DE0A2E0ED938A95E9F79F
:1000440080E4A0E6ED938A95E9F7E8E1F0E0C8954D
:100054003196802DC8953196902D0097B9F0C895AA
:100064003196A02DC8953196B02DC8953196102C97
:10007400C89531966E2F7F2FF02DE12DC8953196BE
:100084000D920197D9F7E62FF72FE1CFEFE9EDBFF6
:10009400C0E7BEC0BA98C29A0895B29902C0E1E01E
:1000A40001C0E0E0E0937000E0917000E03011F1F5
:1000B400E0E4FFE15E166F0620F4E1E0F0E05E0E9E
:1000C4006F1EE2ECF1E0E515F60519F440907000BE
:1000D4000895E0E4FFE1E515F60559F4EAE4FFE1EB
:1000E4005E2E6F2E4424E0917000EC5FE09371006B
:1000F400089507C0442019F0409271004424552407
:10010400662408950A9300917100E0E0E093710081
:10011400E02F09910895AA93EA93FA93EFB7EA932B
:10012400E0917300E0937200E0E0E0937300E093E9
:100134007400A0917500A53028F4E0917500EF5F7C
:10014400E0937500A0917500A53069F4EFEFE0939A
:100154007500E0917200EE5F7E2EE0917200F0E097
:1001640032978E2EB2D0A0917500AF3F79F4B3D000
:10017400EE0FFF1FB5D0A09172007A1620F0A09167
:100184007200A81518F4A7D0E160AAD0E991EFBFD6
:10019400F991E991A99118950A921A92FA926A939F
:1001A4007A938A939A93AA93BA93EA93FA93EFB7BA
:1001B400EA93EEEFE2BFA3E7ED91FD913196FE9352
:1001C400EE93A0917300B0917400AC32E1E0BE07ED
:1001D40041F4E0E0E09375007ED0309711F068942C
:1001E40020F85BDFE991EFBFF991E991B991A99109
:1001F4009991899179916991F9901990099018953B
:10020400C39AE4E1F0E0FA93EA936FD0C3980895B7
:10021400E0E8E6BDE0E0E6BDE6E1E8BBE9E0E7BB37
:10022400E0E0EFBDE4E0E3BFEEEFE2BFE0E0E6BF15
:10023400E9BDE0E4EBBFE2E0E5BFE0E4EABFE2E011
:10024400E9BFE0E8E8B9E0E0E3B924DF78945ADFF5
:100254009E2E992029F1E1E0E915B1F4D1DF20FCCB
:1002640003C050DFE030D9F320FE0EC034D0A0E04C
:10027400B0E056D0E89420F828D0C2DFEEE1F0E0F8
:10028400FA93EA9332D0BCDFE5E0E91549F4A0E043
:10029400B0E0E0E0F0E044D0E0917000E030E1F75D
:1002A40020FE11C0A0E0B0E02CD0A0917600B09167
:1002B4007700EA17FB0721F4E8B3A1E0EA27E8BBDB
:1002C40004D0E89420F8C3CFFFCFE0E0E0937600B9
:1002D400E09377000895E0917600F0917700089517
:1002E400E0937600F09377000895E991F9913096C0
:1002F40039F080E699E00197F1F7A8953197C9F7AD
:100304000895119602D0FE2F1197E199FECFFF9325
:10031400FFB7F894AEBBE09AEDB3FFBFFF91089529
:1003240007D01196EF93EF2F03D0EF911197089513
:10033400E19B02C0A895FCCF9FB7F894AEBBE09AAE
:100344008DB3E81719F0EDBBE29AE19A9FBF0895C7
:00000001FF
